S31508001800D0090020D9180008E7180008E9180008C8
S3150800181000000000000000000000000000000000BA
S315080018200000000000000000000000000119000888
S315080018300000000000000000031900087D380008B9
S31508001840DD450008071900080719000807190008E8
S31508001850071900080719000807190008952800083D
S315080018600719000831260008071900080719000893
S31508001870071900080719000807190008013B00089E
S31508001880553B00080000000000000000071900088A
S3150800189000000000071900080719000807190008C2
S315080018A0000000000719000807190008E53E0008AF
S315080018B007190008071900080719000800000000A2
S315080018C0EE11AA550348854600F0BEFB00480047BE
S315080018D029580008D00900200B4880F308880B48CF
S315080018E080470B480047FEE704207146084202D0AD
S315080018F0EFF3098001E0EFF30880714603F05CFE20
S31508001900FEE7FEE7FEE7FEE7D0090020953A000865
S31508001910C518000830B50B460146002020220124D0
S3150800192009E00D46D5409D4205D31D469540491B05
S315080019302546954040191546521E002DF1DC30BD4E
S3150800194070B500242546002801DA01244042002902
S3150800195001DA01254942FFF7DDFFAC4200D04042DB
S31508001960002C00D0494270BD03460B439B0703D0A9
S3150800197009E008C9121F08C0042AFAD203E00B7846
S315080019800370401C491C521EF9D27047D2B201E0BE
S315080019900270401C491EFBD270470022F6E710B5BC
S315080019A013460A4604461946FFF7F0FF204610BDBF
S315080019B0F8B502464A40D40F42004B0052085B086D
S315080019C09A4202D20246084611464A0023D0C30D5F
S315080019D04A00DDB2120EAD1A202D35DA490201266B
S315080019E0490AF6058A19002C00D0524220214F1BBD
S315080019F01146B9402A411018C20D9A4221D0002C2E
S31508001A0017D0012D08DCDA05801AD20F8019D20703
S31508001A10DBB200F081FAF8BDDA05801A012340002E
S31508001A201B06C01880185A428018CA0F104349006E
S31508001A3007E04908C2071143DA05801A80194008E9
S31508001A40801800F061FAF8BD61000122511A001BE6
S31508001A50F7E70122D2075140AAE70122D2075040F0
S31508001A60A6E7024670B54A40D30FDB0740002DD0E3
S31508001A704A002AD0010E140E000212020919400A61
S31508001A80520A8418E50104465443000A120A2E0431
S31508001A905043A4194219200CC543AA18120C012553
S31508001AA0AD03521C521912047F39240400D0521C6B
S31508001AB0104301D44000491EC2B20C06C0092018C2
S31508001AC0401C4008802A02D003E0002070BD400870
S31508001AD04000002900DA0020184370BD70B50246A0
S31508001AE04A40D50F40004A00ED0740085208002832
S31508001AF014D0002A12D0C40DD30D41020120C0050E
S31508001B005202490A520AE41A091812187D349142F7
S31508001B1001D3641C00E04900002C01DA002070BDE6
S31508001B200023914201D3891A03434008490000283B
S31508001B30F7D100290AD0914202D10121C90705E04F
S31508001B40914201D2012101E00121C943E005C018F3
S31508001B50401900F0D9F970BDF0B507460846584057
S31508001B6087B0C00F049048000E465900400849083F
S31508001B70BC1A884105D2384631461E4617460B46DA
S31508001B8002465800400810434CD0300D03904005DB
S31508001B905900400D490D0590401A0290402872DA06
S31508001BA018030121000B09050843019004980092C7
S31508001BB0002805D0019952420020884100920190E0
S31508001BC0029840210A1A0199009800F069F9054619
S31508001BD00C466B4607CB00F084F9C0197141039A8D
S31508001BE00E0D0023D71756401A467A40164344D09E
S31508001BF0049A002A2DD0029A012A039A15DC1205A6
S31508001C00C01A914101263605001C7141D20F059E66
S31508001C10D2070093019202962A46234600F0C2F99B
S31508001C2007B0F0BD38463146FAE71605224A0F4690
S31508001C30B218C01AB74101210905001C4F41001806
S31508001C407F41114618187941E20F10436D19644116
S31508001C5013E0E2076D0815436408C2071443039AA4
S31508001C6001261205C01A91413605001C7141CE079E
S31508001C70400830434908C01851412A46234600F017
S31508001C8084F9CDE7FFE7049801224000C117121A2C
S31508001C9000238B4104983146C417381AA141EEE750
S31508001CA030B40124E407634030BC55E730B401245E
S31508001CB0E407614030BC4FE70000E0FFF0B51FB411
S31508001CC088B00B990998002448400999C00F490023
S31508001CD049080991C0070B990090490049080B91DA
S31508001CE009990898A64608431CD00B990A980843F0
S31508001CF018D0099801244000420D4800410D099862
S31508001D0024050003000B204309900B980003000BE1
S31508001D1020430B9050181C49401800220190144685
S31508001D20104605E0002001460DB0F0BD032801DA93
S31508001D30034600E003239C46C11A0AAE0AE05F0088
S31508001D4008ADED5B4F00F75B7D430027AA187C4181
S31508001D50491C5B1E6145F2DD410004AB5A52210461
S31508001D60120C0A43240C401C0828DFDB0198029059
S31508001D700099704601910090059B049A0799069868
S31508001D8000F010F9D0E700000DFCFFFF10B50022A7
S31508001D909623114600F0C0F810BD4100400201220A
S31508001DA0400AD205090E80187F2901DA00207047FB
S31508001DB0962903DC9622511AC840704796398840FE
S31508001DC0704700004A0009030123090B1B05194344
S31508001DD0094B10B5520D9A4201DA002010BD064B88
S31508001DE034339A4203DC9A1A00F06AF810BD0349A4
S31508001DF05118884010BD0000FF030000CDFBFFFF0F
S31508001E00C20FD207400040080BD0C10D0723DB01E3
S31508001E10C91840020905400A1143C2084007114380
S31508001E20704700200146704710B5002904DB0124DD
S31508001E30E40740428C412146002B04DB1C46012363
S31508001E40DB075242A3418B4200D1824210BD0000FB
S31508001E5010B5002904DB0124E40740428C412146E1
S31508001E60002B04DB1C460123DB075242A34199429F
S31508001E7000D1904210BD00000122D207002800DBE5
S31508001E80101A002900DB511A814270470122D20735
S31508001E90002800DB101A002900DB511A8842704717
S31508001EA010B5202A04DB0146203A9140002010BDD7
S31508001EB0914020239C1A0346E3401943904010BDE5
S31508001EC010B5202A04DB0846203AD040002110BD70
S31508001ED00B46D340D0402024A21A91400843194605
S31508001EE010BD10B5202A06DBCB170846203A10414C
S31508001EF0C1170B4306E00B461341D0402024A21A13
S31508001F0091400843194610BD002904DA401C4900CF
S31508001F1001D140084000704770B40024050C05D173
S31508001F201024000402D1002921D01124050E01D164
S31508001F3000020834050F01D10001241D850F01D1C7
S31508001F408000A41C002801DB4000641C002908D07E
S31508001F5020252E1B0D46F540A14000D0012129431E
S31508001F60084301061B1B000ADB1D02D5002070BCB6
S31508001F707047DB05181880180029F8DA401C490054
S31508001F80F5D170BC40084000704710B5002B08DA40
S31508001F900024401C614192185B411A4301D1400854
S31508001FA0400010BDF0B51FB482B005460C0003D042
S31508001FB0084602F045FB02E002F042FB20300246EA
S31508001FC0009021462846FFF76BFF049B059A0446B6
S31508001FD00F4618431143084314D0184610431BD024
S31508001FE0009840210A1A18460599FFF769FF054621
S31508001FF00E46009A05990498FFF752FF084305D044
S31508002000012004E02046394607B0F0BD0020C1177C
S3150800201005430E432C43374300990E986305401A2F
S315080020207905E40A00220C43FD0A0A3002D500208D
S315080020300146E9E70105101969410C9C0D9D001937
S315080020406941FFF7A2FFDFE7064C0125064E05E0CA
S31508002050E36807CC2B430C3C98471034B442F7D3BB
S31508002060FFF734FC94670008B467000810B5044607
S31508002070002C08D101210920C00600F071FE0020BD
S3150800208000F0AAF852E0012C05D102210920C00669
S3150800209000F066FE4AE0022C05D104210920C0069C
S315080020A000F05EFE42E0032C05D108210920C00697
S315080020B000F056FE3AE0042C05D110210920C0068E
S315080020C000F04EFE32E0052C05D120210920C0067D
S315080020D000F046FE2AE0062C05D140210920C0065C
S315080020E000F03EFE22E0072C05D180210920C0061B
S315080020F000F036FE1AE0082C04D101210D4800F044
S315080021002FFE13E0092C04D102210A4800F028FE0C
S315080021100CE00B2C04D11021064800F021FE05E046
S315080021200C2C03D18021034800F01AFE204600F04B
S3150800213053F810BD000400487FB5002000900190B8
S315080021400290039000241BE000250CE0E8000E49ED
S3150800215040186100405AA1006A4651584018A1002B
S315080021605050681C85B2142DF0DBA1006A46505801
S315080021701421FFF7CFFB6100044A5052601C84B259
S31508002180042CE1DB7FBD0000280400205401002058
S3150800219000B587B001A800F0AFF80121480201F0A8
S315080021A0DFF90020019030200290012040020390C0
S315080021B000200690059001A9064800F031F8012193
S315080021C0044800F021F80121024800F011F807B090
S315080021D000BD00000024014010B504460723002274
S315080021E02146024800F038F810BD000000240140DE
S315080021F0002904D0426801231A43426003E042687A
S315080022005208520042607047002904D082680823A9
S315080022101A43826003E0826808239A438260704703
S3150800222042680B4B1A4042600B684A681A43436877
S315080022301A4342608268074B1A4082600B694A69F2
S315080022401A438B681A4383681A43826070470000F2
S315080022500FBCFFFF8FF1F9FFF0B504460D46164691
S315080022601F463F073F0F2B46082B0FD91B071B0F8F
S31508002270083B606F9A000F21914088436067606F42
S3150800228099003A468A40104360670BE0206F9A002F
S315080022900F21914088432067206F99003A468A406B
S315080022A010432067E0680121A9408843E060E068A0
S315080022B00121A9400843E060012080032840002846
S315080022C003D0012000F020F807E00120C0032840D1
S315080022D0002802D0012000F017F8F0BD002905D02B
S315080022E08268FF2301331A43826004E08268FF2371
S315080022F001339A4382607047002101604160816022
S315080023000173016141617047002806D00649496892
S315080023100C221143044A516005E0034949680C221E
S315080023209143014A516070470024014010B509489D
S315080023300078002809D0FFF7FFFE0020054908703D
S3150800234000F058FD0121044881767E2002F052F9FA
S3150800235010BD00005C01002044030020FFB583B0D7
S315080023600C46029400200190002726E000261CE077
S31508002370721C039951430846791CFFF7CBFA0546A8
S31508002380A54201D9281B00E0601B05460298A84211
S3150800239004D90295059806700698077002980028D1
S315080023A002D10120019002E0761C402EE0D300BF46
S315080023B00198002800D002E07F1C042FD6D300BF66
S315080023C0029807B0F0BD000000BF00BF00BF00BF05
S315080023D000BFBFF34F8F00BF00BF00BF06480749C5
S315080023E0C86000BF00BF00BFBFF34F8F00BF00BF6C
S315080023F000BF00BF00BFFDE70400FA0500ED00E0DE
S3150800240010B500F001F810BD10B523480078002873
S3150800241017D1224801F02CF901283CD11F48007831
S31508002420002838DD1D480078402834DC01F02DFDF1
S315080024301B490860012018490870002019490870CE
S3150800244029E0164A17490978491C501801F010F96D
S31508002450012816D113480078401C124908700F4805
S3150800246000780978884216D100200B4908700B4875
S315080024704078FF280FD10B48007802280BD1FFF7C8
S31508002480A3FF01F002FD064909686431884202D9B2
S3150800249000200149087010BD29010020AC03002066
S315080024A02C0100202801002078B50246002327E0E9
S315080024B0002020E08400155B441CA400145BA542A0
S315080024C018DD8400A5182E886C4626806D886580E0
S315080024D08400A518441CA400A41826882E806488A5
S315080024E06C80441CA400A5186C4624882C806C4675
S315080024F064886C80401C4C1EE41A8442DADC5B1C3F
S315080025004C1E9C42D4DC78BD10B586B00446012129
S31508002510880301F025F80121880401F001F8032257
S315080025201146224800F007FC032204211F4800F048
S3150800253002FC01A801F07BFD019430216846018167
S3150800254000214181818101821821C18101A9184890
S3150800255001F02AFD0121164801F003FD05A800F047
S3150800256040FC082168468182012181751821C175C0
S3150800257005A90E4800F092FB102168468182482181
S31508002580C17505A9094800F089FB1B216846017039
S31508002590032141700121817000F070FF01220221A0
S315080025A0034801F0F6FC06B010BD00000004004820
S315080025B00038014070B502460B46FF25FF2408E0A7
S315080025C01178521C69400748405C60400546064839
S315080025D0445C18465E1EB3B20028F1D12802204397
S315080025E070BD000094650008946600080146002244
S315080025F00E4B1A61CA005A6100229A6105221A61B5
S3150800260000BF0A4A1069C207D20F002A04D0012265
S3150800261012040240002AF4D0044A126952085200F1
S31508002620024B1A6100229A617047000000E000E040
S3150800263010B500210848FFF751FE022000F052F8B5
S3150800264001200649087001020920C00600F0C5FBF2
S3150800265002F068F810BD0000002401406401002063
S3150800266000B589B00121084600F05AFF1A4800F063
S3150800267045F801A800F08EF818480190184802900D
S31508002680002168460173042004906846017580217C
S3150800269041754900C182890001832021817609029A
S315080026A081830021C183018401A90B4800F04CF8FD
S315080026B00121094800F01CF801220221064800F011
S315080026C039F809216846017002214170012181709B
S315080026D000F0D4FE09B000BD080002400024014005
S315080026E0F0030020014948607047000000000240DE
S315080026F00268520852000A430260704710B5044641
S315080027002068400840002060002020606060A060CB
S31508002710E060E1B2084608380521FFF7FBF80146F4
S315080027200F2088400249496808430149486010BD9E
S3150800273000000240002A03D003680B43036002E04E
S3150800274003688B430360704710B50A7A8B7D1A437A
S315080027500B7C1A434B7C1A434B8A1A438B8A1A43BF
S315080027600B8B1A434B8B1A430368094C23401A43B5
S31508002770026002680123DB039A438B8B1A430260CB
S31508002780CA6842600A6882604A68C26010BD000072
S315080027900F80FFFF0021016041600172C160017472
S315080027A041744182818281750183418381837047A7
S315080027B070B506460C4621460A4800F00FFA05464B
S315080027C0002D01D1401E70BD0648854202D106483B
S315080027D0051B00E02D1B224629463046FFF7C4F8A4
S315080027E02046F0E700F4000800FC000870B506462D
S315080027F00C4621460A4800F0F1F90546002D01D19C
S31508002800401E70BD0648854202D10648051B00E0F9
S315080028102D1B224629463046FFF7A6F82046F0E744
S3150800282000F0000800F8000870B506460C46214678
S315080028300A4800F0D3F90546002D01D1401E70BDA7
S315080028400648854202D10648051B00E02D1B224694
S3150800285029463046FFF788F82046F0E700F80008D2
S315080028600000010870B505460C462246024928466E
S3150800287000F075F9204670BD00F4000870B50546ED
S315080028800C4622460249284600F069F9204670BDE2
S3150800289000F0000810B5024800F004F810BD00006A
S315080028A0208000000149486170470000000401408B
S315080028B01CB5684600F0A9F80F21002000F07CF846
S315080028C00120C00300900021684601711021417162
S315080028D00121817100F010F80521002000F06CF844
S315080028E020200090002168460171102141710121C4
S315080028F0817100F001F81CBD8179002948D02D4965
S315080029000968026891432B4A1160114649680268B2
S315080029109143284A51600179002906D11146096870
S3150800292002681143234A116005E022494968026892
S315080029301143204A51601F498968026891431D4A1C
S3150800294091601146C968026891431A4AD160417973
S3150800295010290CD11146896802681143154A9160FD
S315080029601146C96802681143124AD16020E04179CC
S31508002970082906D10F498968026811430D4A9160F2
S3150800298016E00C49C968026811430A4AD1600FE08B
S315080029900179002906D10749096802689143054A61
S315080029A0116005E00349496802689143014A51608C
S315080029B0704700000004014010B50D4A8B109B00BB
S315080029C0D3588A07140F0F22A2409343084A8C1043
S315080029D0A40013518B109B00D2588B071C0F03467B
S315080029E0A3401A43024B8C10A4001A5110BD0000D4
S315080029F00800014008B507216846017002214170A8
S31508002A000121817000F03AFD08BD002101600171C5
S31508002A100C214171002181717047000010B50446F0
S31508002A2008480069022108430649086108464461C6
S31508002A3000694021084303490861034800F00EF97C
S31508002A4010BD000000200240FF0F00000C48C068BF
S31508002A50C007C00F002801D0012070470848C06889
S31508002A6004210840002801D00220F6E70448C0687F
S31508002A7010210840002801D00320EEE70420ECE7E7
S31508002A800020024003480069802108430149086183
S31508002A90704700000020024030B504460D46054840
S31508002AA00069012108430349086125800F2000F0C9
S31508002AB0D5F830BD0020024010B57E2001F09AFD01
S31508002AC0064800F00FF87E2001F094FD044800F057
S31508002AD009F87E2001F08EFD10BD000000F4000804
S31508002AE000F0000810B5044600F0ACF82046FFF7E1
S31508002AF095FFFFF7C7FF10BD70B5034601250022F5
S31508002B0008E050001C5A0748844201D0002506E018
S31508002B10501C82B2CE0F761876109642F1DC00BFB2
S31508002B20284670BDFFFF0000F8B505460E46144658
S31508002B3000F088F87E2001F05DFD002707E029886F
S31508002B403046FFF7A9FFB61CAD1C781C87B2E10F0B
S31508002B5009194910B942F2DCFFF794FFF8BDF8B538
S31508002B6007460C4615462946204600F037F806461D
S31508002B70002E0DD12046FFF7B5FF01208002201850
S31508002B80FFF7B0FF2A4621463846FFF7CDFF24E077
S31508002B90012080022018401BB0420AD10120800281
S31508002BA02018FFF79FFF2A4631463846FFF7BCFF35
S31508002BB013E00120C0022018401BB04208D120466D
S31508002BC0FFF790FF2A4631463846FFF7ADFF04E087
S31508002BD02A4631463846FFF7A7FFF8BDF8B5054639
S31508002BE00E462F46E807C00F002801D000BFFEE7B3
S31508002BF031460120C002FEF7A3FE002901D000BF1E
S31508002C00FEE700240BE02046704347193146384654
S31508002C10FFF772FF012800D108E0601C84B2314634
S31508002C200120C002FEF78CFEA042ECDC00BF314654
S31508002C300120C002FEF784FEA04200D100273846D4
S31508002C40F8BD0000024803494860034848607047D9
S31508002C502301674500200240AB89EFCD10B5024637
S31508002C6000BFFFF7F3FE0346521EFF2400E0641E72
S31508002C70002CFCD1012B01D1002AF2D106480069AB
S31508002C8077218843044908613420C860002A01D1A5
S31508002C90052010BD1846FCE700200240F8B502469C
S31508002CA0CD782F073F0FCD7810263540002D01D05F
S31508002CB08D782F431446002011E085062B0E0D88CB
S31508002CC0012686403540002D07D025680F269E40F0
S31508002CD0B5433E469E4035432560451CE8B2082864
S31508002CE0EBDB141D0D882D120095002011E08506DA
S31508002CF02B0E01258540009E3540002D07D02568FE
S31508002D000F269E40B5433E469E4035432560451CEA
S31508002D10E8B20828EBDBCD78282D04D155690E8852
S31508002D203543556106E0CD78482D03D115690E88DF
S31508002D3035431561F8BD70B54D07EB0E082902DA63
S31508002D400546203501E0054624352C460F269E40CB
S31508002D502568B54316469E403543256070BD00007C
S31508002D6038B504460D460920C006844203D1012120
S31508002D70480400F0D5FB1148844203D10121000222
S31508002D8000F0CEFB0E48844203D10121000200F078
S31508002D90C7FB0C48844203D10121080500F0C0FB9B
S31508002DA0684600F01EF868460580012181700021FA
S31508002DB0C17069462046FFF771FF38BD0004004818
S31508002DC000080048000C00480246906808400028A1
S31508002DD001D0012070470020FCE74161704701617E
S31508002DE070470021C9430180022181700421C17006
S31508002DF070470000F0B58BB0002009900890079046
S31508002E0006907E2001F0F6FB002611E07100D14AFB
S31508002E10505AFEF7BBFF0546CF49FEF75FFE04464C
S31508002E20CE49FEF71EFEB100CD4A5050701C86B240
S31508002E30042EEBDBCA4A51689068FEF70AFE044680
S31508002E40C849FEF74BFE0990C54948680999FEF737
S31508002E5045FEC5490860C549C3480068FEF701FE36
S31508002E600446FEF79AFF81B2C1488184FF38893843
S31508002E70807B00283BD1BF498889FEF787FFBD497B
S31508002E800490C888FEF782FFBB490390FEF726FE2A
S31508002E9007460499FEF7E5FD0546B449FEF71EFE0A
S31508002EA00446B4498889FEF771FF0746AF49FEF71D
S31508002EB015FE0546AC4801682846FEF7CEFD2146B4
S31508002EC00590FEF70BFE0790AA494889FEF75EFFB4
S31508002ED005460799FEF76CFD0446FEF75EFFA7490F
S31508002EE008600846008881B2A148018235E0A048FA
S31508002EF0007E002831D19F481038C078012828D193
S31508002F0099480068FEF77CFF04469D4A9D4BFEF7EC
S31508002F109FFF1BD294480068FEF772FF04469A4A40
S31508002F209A4BFEF781FF11D290498F480068FEF749
S31508002F3098FD0446FEF731FF81B28E48818101462D
S31508002F40888902F0B3FD02F031FA02E0022002F0AD
S31508002F507BFE002187481038817386481038C07B6D
S31508002F60012805D102F022FA002182481038C173DF
S31508002F707F4820308079012809D17E4B5A89998962
S31508002F80D88802F0EBFD0021794820308171784914
S31508002F90088AFEF7FBFE7E49086071498868FEF7D5
S31508002FA02FFF0446764A52427A4BFEF7D5FD002299
S31508002FB0794B01910090FEF781FE002201239B07C1
S31508002FC003910290FEF77AFE05910490FEF7FAFE49
S31508002FD081B26748C181FF38C1380088FF21F531C1
S31508002FE0884275DD0020634948390880084638302C
S31508002FF0C07801283FD15E48007E00283BD058495A
S3150800300088686649FEF72DFD0446FEF7C6FE85B2BA
S31508003010534948686149FEF724FD0446FEF7BDFE9C
S3150800302080B2281A032810DA52484838C068AF21F7
S315080030308900884209D94E48407A002805D14D4969
S315080030404839C86004214A484172454988680021C0
S31508003050FEF712FF05D0424948680021FEF70CFF2B
S3150800306009D14348407A002805D142494839C86001
S3150800307005213F4841723A49C868FEF7C1FE044631
S31508003080474A484BFEF7D0FE23D23549C868FEF7B3
S31508003090B7FE0446444A454BFEF7C6FE13D2202126
S315080030A04348FFF791FE00280DD13148007A0128E0
S315080030B009D12F48407A002805D12E494839C860D9
S315080030C006212B48417201212A481038417013E025
S315080030D03DE02349C8683749FEF7D8FE0CD2244894
S315080030E0007E002804D1002122481038417003E0F0
S315080030F001212048103841701949C8682E49FEF741
S31508003100C5FE04D201211B481038017103E00021D5
S31508003110184810380171174810384078002810D11F
S315080031201348007A012805D1C1020920C006FFF715
S3150800313054FE0CE00121C9020920C006FFF74FFE24
S3150800314005E00121C9020920C006FFF748FE0BB0B9
S31508003150F0BD00005401002000F07F450000A040AB
S31508003160180400203333A3406801002000007A4485
S3150800317044030020CC01002000247449700100207B
S31508003180666666666666E63FCDCCCCCCCCCCEC3FB4
S315080031906C0300209999B93F000059400000C842C5
S315080031A0A245B6F3FDD4EC3F75931804560EDD3FE1
S315080031B00004004852B89E3FFCA9794001480068BF
S315080031C07047000038010020034800680349097861
S315080031D04018014908607047380100204001002066
S315080031E008B50121480400F09BF90121880400F084
S315080031F097F96846FFF7F5FD0421684601804821DE
S31508003200C17069460920C006FFF748FD6846FFF702
S31508003210E8FDFF210131684601804821C1706946F1
S315080032200748FFF73BFD6846FFF7DBFD20216846A8
S3150800323001800421C17069460148FFF72FFD08BDCA
S315080032400004004810B504210920C006FFF7BCFD9C
S3150800325000286AD05A48407B00285BD15848007A33
S31508003260012839D15648007E002835D155480078BE
S31508003270401C544908700846007805281FDB0020C2
S3150800328008704F487838408900280AD14E484F4977
S31508003290C86001214D483830C172FF301130418174
S315080032A00AE0022149483830C17200204749C860FF
S315080032B0002143487838418101F0A4F90CE04148DF
S315080032C00078022808DC4148C0687D210901884247
S315080032D002D900203D49C8603948007E002816D129
S315080032E03A48C0693A49884211D3354878384089FE
S315080032F0002805D137483549C8610020C86006E06E
S3150800330030480078022802DC00203049C8600121D4
S315080033102B4841733048007800280DD101202E49EA
S31508003320087001212648017306E000202A49087022
S315080033300021234801734173244800697D21C9008F
S31508003340884237D900202149086100211C480173A9
S31508003350007E002828D11A4878384088032829DAB8
S31508003360174878384089002824D118483830007919
S3150800337000280ED11248007A01281BD101211048D5
S31508003380017600201149C860012110483830C17201
S3150800339010E00B48407A00280CD1012108484172F8
S315080033A000200A49C86005E000200849C8600021D5
S315080033B0034801727E2001F01DF90148007B10BD0B
S315080033C044030020C4000020DC050000840100201E
S315080033D030750000606D00007E01002008B50121EF
S315080033E0480400F09DF80121880400F099F8684621
S315080033F0FFF7F7FC40216846018001218170102102
S31508003400C17069461B48FFF749FC1B49684601809D
S31508003410012181701021C17069460920C006FFF795
S315080034203DFC02220D210920C006FFF784FC01217C
S31508003430090368460180012181701021C17069461F
S315080034400920C006FFF72AFC08210920C006FFF755
S31508003450C6FC20210920C006FFF7C1FC102109205F
S31508003460C006FFF7BCFC012109030920C006FFF7C7
S31508003470B4FC08BD00040048398900008178002999
S3150800348025D0174903221202891802789210920051
S31508003490895802789207D30EFF229A4091434278C0
S315080034A09207120E03789B07DB0E9A4011430C4ACB
S315080034B003231B02D21803789B109B00D150017876
S315080034C0CA06D20E01219140054A116007E001782B
S315080034D0CA06D20E01219140014A80321160704716
S315080034E000E100E009480A494860002048875A2058
S315080034F088870887074808630020C8620648486224
S31508003500064888620448C8617047000000003443D2
S315080035106C0300209A99993E000020410000484219
S31508003520002905D0054A52690243044B5A6104E052
S31508003530024A52698243014B5A61704700100240A1
S31508003540002905D0054AD2690243044BDA6104E032
S31508003550024AD2698243014BDA6170470010024081
S31508003560002905D0054A92690243044B9A6104E092
S31508003570024A92698243014B9A61704700100240E1
S3150800358010B500F031F804494968F02211400909DC
S31508003590024A515CC84010BD0010024004010020D8
S315080035A010B5FFF7EDFF05494968072212021140D9
S315080035B0090A034A515CC84010BD000000100240C9
S315080035C00401002010B5FFF7DBFF0549496807220B
S315080035D0D2021140C90A034A515CC84010BD000016
S315080035E00010024004010020F8B51E4840680C216E
S315080035F00840042802D008282ED101E01A4C2DE0F4
S31508003600184840300069C007C00F00280AD015487E
S315080036104030006902210840002801D0134802E022
S31508003620114800E0104807460E4840300069FF215F
S3150800363009040840000C451C0A4840300069072167
S3150800364009020840000A461C3946694308463146BD
S31508003650FEF760F9044601E0034C00BF00BF2046B0
S31508003660F8BD00000010024000127A0000093D0073
S3150800367070B5044600250221074800F078FC0028AA
S3150800368008D0054800F0CCFC20700221024800F062
S3150800369066FC0125284670BD0038014010B500F0CB
S315080036A001F810BD00B585B06248006801210843DD
S315080036B06049086000BF5F4800680221084000288A
S315080036C0F9D05D485D4908605D48006810210843E7
S315080036D05B49086008460068C008C000086057498A
S315080036E00968481E5749FEF715F9049054480068BA
S315080036F004994907490F0843514908604D484068ED
S31508003700514908404B49486008464068902108439B
S31508003710484948600846406848604848006846493D
S31508003720884207D9434840680521090208434149A8
S3150800373048600BE0414800684449884206D93D483C
S3150800374040680121890208433A4948606B4601AA44
S315080037503A4801683E48FEF701FE3648403000699F
S3150800376080088000334940310861084600694008EE
S3150800377040000861684600784007400F0290684696
S3150800378000794006400E03902A48C0698905084317
S315080037902849C8612748403000692E49084025490C
S315080037A04031086103980004029909020843214937
S315080037B04031096908431F49403108611D480068BE
S315080037C00121090608431B49086000E000BF1948A3
S315080037D000680121490608400028F7D015484068C6
S315080037E0800880001349486008464068022108435B
S315080037F01049486000E000BF0E4840680C210840A8
S315080038000828F8D10120FEF7F1FE0A484068102181
S315080038108843084948600120FEF7E8FE05484068E5
S3150800382080218843034948600120FEF7DFFE05B082
S3150800383000BD00000010024000A24A041401002046
S315080038400020024000366E010FC0FFFF005125021E
S3150800385000127A00FFF800FF042806D10649096914
S3150800386004221143044A116105E003490969042247
S315080038709143014A1161704700E000E010B5FFF777
S31508003880A3FC7B480088401C794908800846C06824
S31508003890401CC86077480088401C764908807648EE
S315080038A00068002804D074480068401E7249086001
S315080038B07248007B012805D16D480069401C6C4997
S315080038C0086102E000206A49086169483830007AD0
S315080038D001280ED166484069401C6549486108467A
S315080038E040696749884207D9002161483830017222
S315080038F002E000205E4948615D483830807A012838
S3150800390005D15B48C06A401C5949C86202E00020DC
S315080039105749C8625948007E002809D0544840686B
S31508003920401C534948600846806A401C886203E088
S3150800393000204F49486088625048807A04280AD196
S315080039404B48C0694F49884208D24948C069401C5B
S315080039504749C86102E000204549C861FF21013195
S315080039604948FFF731FA002813D0414838304078E3
S3150800397000280ED14148007A01280AD13C48006A3D
S315080039803F49884208D23A48006A401C38490862CA
S3150800399002E000203649086235483830C07A0128E6
S315080039A013D1C1030920C006FFF719FA3048816808
S315080039B08068401C2E4A9060FF20F530814225D948
S315080039C0002110463830C17220E029483830C07AC4
S315080039D0022812D181030920C006FFF700FA2448FD
S315080039E081688068401C224A9060284881420DD927
S315080039F0002110463830C17208E000201C49886052
S31508003A000121C9030920C006FFF7E7F91B48007E14
S31508003A10012805D11648006B401C1549086302E0C9
S31508003A200020134908637E2000F0E4FD2021164893
S31508003A30FFF7CAF900280AD00D48406A1449884297
S31508003A4008D20B48406A401C0949486202E0002037
S31508003A50074948620948407E012805D10448406B59
S31508003A60401C0349486302E000200149486310BD31
S31508003A708401002030010020340100204403002086
S31508003A808813000050C3000000040048DC0500004D
S31508003A90B888000010B51648006801210843144983
S31508003AA008600846406813490840114948600846B6
S31508003AB00068114908400E49086008460068012157
S31508003AC0890488430A49086008464068C3210904EE
S31508003AD08843074948600846006808490840044979
S31508003AE008609F2000048860FFF7D8FD10BD00001D
S31508003AF0001002400CC0FFF8FFFFF6FEFFFF8F0024
S31508003B0010B50421080700F01DF9002806D0042185
S31508003B10080700F0F1F801210148817010BD000086
S31508003B20BC01002008B501214804FFF7F9FC022270
S31508003B3001210920C006FFF7FEF802216846018028
S31508003B401821C1700121817069460920C006FFF756
S31508003B50A5F808BD10B50121194800F0F3F80028AA
S31508003B602CD00121164800F0C7F81648807801289D
S31508003B7024D11548C17AC07A401CC2B21248C27212
S31508003B800B291BDD0F48C078012803D00E48407E5C
S31508003B90012805D1FF2101310920C006FFF71FF9C9
S31508003BA00948C07A0D2809DD0021064881700121DF
S31508003BB00648FEF793FB00210348C17210BD0000BA
S31508003BC000040040BC0100204403002000240140FA
S31508003BD030B589B004460D4601210846FFF7B0FC0A
S31508003BE006A800F049F90794684605830021018470
S31508003BF008A881706846817606A90120800700F02A
S31508003C0005F90F216846017101214171817101A8E9
S31508003C10FFF734FC0421080700F06AF801220421A2
S31508003C20080700F09CF802A800F0DCF86021684656
S31508003C300172012141720020039000216846017437
S31508003C4002A90120800700F095F80821C80600F0AF
S31508003C50C1F84021080600F06DF80121880700F038
S31508003C603BF80121880700F057F80121880700F082
S31508003C7047F809B030BD00007FB504460D4601215E
S31508003C800220FFF75DFC684600F0F6F801946846E6
S31508003C900580002101818172817069460D4800F016
S31508003CA0B5F8102168460173022141730121817319
S31508003CB003A8FFF7E3FB0121064800F019F80122E3
S31508003CC01146044800F04BF80121024800F018F8A4
S31508003CD07FBD000000040040002904D0026880234C
S31508003CE01A43026003E0026880239A430260704721
S31508003CF002698A430261704702698A430261704712
S31508003D00002904D0026801231A43026003E002680E
S31508003D105208520002607047002905D0426C012300
S31508003D20DB031A43426404E0426C0123DB039A4333
S31508003D3042647047826907231B039A430B021A439E
S31508003D4082617047024610690840002805D0D0688D
S31508003D500840002801D0012070470020FCE7002A0F
S31508003D6003D0C3680B43C36002E0C3688B43C360D8
S31508003D707047000010B5826907231B039A430B7826
S31508003D801B021A4382610A7A12014B781B011A43F5
S31508003D90036A3024A3431A4302624A6882630C4AC0
S31508003DA0904213D14A7A12018B781B011A43036A8F
S31508003DB0C024A3431A4302624A8992008B899B0056
S31508003DC01A4343682401A3431A43426010BD000006
S31508003DD0002C014082690123DB029A430B021A4335
S31508003DE082617047002101704170817041600172E3
S31508003DF0417241818181704701229207904201D127
S31508003E00816301E08AB28263704700000268032377
S31508003E101B029A430B891A430260134A904206D042
S31508003E2001229207904202D0104A904205D10268B8
S31508003E3070239A438B781A4302600B4A904205D046
S31508003E400B4A904202D00B4A904205D1026B120AE5
S31508003E5012028B7A1A4302634A68C2620A8882622D
S31508003E600122426170470000002C01400004004016
S31508003E7000440140004801400021C9434160002137
S31508003E800180018181708172704710B5FFF796F93C
S31508003E9010BD000070B5FFF773FB05467D21C9000C
S31508003EA0FDF738FD0446601E0C49884200D90CE02F
S31508003EB0601E0B4948610321081F00F0E7FB00203C
S31508003EC0074988610720086100BF0420FFF7C4FC82
S31508003ED00021481E00F0DAFB70BD0000FFFFFF005E
S31508003EE000E000E010B502210A4800F049F8002871
S31508003EF00ED0084800F094F8C4B20748407A002863
S31508003F0002D1204601F08EFA0221024800F027F875
S31508003F1010BD000000380140BC01002010B5044661
S31508003F202146054800F080F800BF0121024800F04C
S31508003F301EF80028F9D010BD0038014070B50446B7
S31508003F400D467E2000F056FB03E02078641CFFF740
S31508003F50E5FF2846691E8DB20028F6D170BD41617D
S31508003F6070478269520852000A43826170470246C6
S31508003F7090680840002801D0012070470020FCE71F
S31508003F800246D0680840002801D00120704700206A
S31508003F90FCE7002A03D003690B43036102E00369C7
S31508003FA08B4303617047000070B504460D46002632
S31508003FB0E0693021884329790843E061E0694421B2
S31508003FC08843A9790843E061E06980088000297A76
S31508003FD00843E061A0691821884369890843A061FC
S31508003FE0A06904218843297B0843A0610B488442C1
S31508003FF003D1FFF7E7FA064602E0FFF7D1FA0646CD
S3150800400030462968FDF786FC000920623046296893
S31508004010FDF780FC0007000F606270BD00380140A4
S3150800402001464868C0B27047CAB2026070474B2161
S31508004030C9010160302101710021817101721821C5
S31508004040418100210173704710B51F48807E012801
S3150800405039D11D4878384088030000F008FB05046C
S31508004060111E2B2C2D001848C089FF219B31884230
S3150800407005DC012114487838418000F0C3FA1BE0BA
S315080040801148C089FF217831884205DC02210E4893
S315080040907838418000F0B6FA0EE00B48C089FF2157
S315080040A05F31884205DC032107487838418000F0F3
S315080040B0A9FA01E000E000BF00BF0348007A002823
S315080040C001D100F09FFA10BD4403002010B57948CD
S315080040D04088002806D0012848D0022877D003282F
S315080040E043D1A0E0022173487830817220217248BA
S315080040F0FEF76AFE002829D07049C868FF21F53105
S31508004100FDF708FCC007C00F00280FD110210920B1
S31508004110C006FEF762FE08210920C006FEF75DFE0E
S3150800412020210920C006FEF758FE1EE010210920AE
S31508004130C006FEF754FE08210920C006FEF74FFE0A
S3150800414020210920C006FEF74AFE0EE010210920AC
S31508004150C006FEF742FE08210920C006FEF73DFE0E
S3150800416020210920C006FEF738FEA0E001215148AB
S315080041707830817220215048FEF726FE002815D097
S315080041804E49C868FF21F531FDF7C4FBC007C00FCB
S31508004190002805D108210920C006FEF71EFE0AE000
S315080041A008210920C006FEF71AFE04E008210920A6
S315080041B0C006FEF712FE10210920C006FEF70FFE04
S315080041C020210920C006FEF70AFE70E0FFE720213D
S315080041D03948FEF7F9FD002815D03849C868FF2187
S315080041E0F531FDF797FBC007C00F002805D1102150
S315080041F00920C006FEF7F3FD0AE010210920C006D3
S31508004200FEF7EBFD04E010210920C006FEF7E5FDE8
S3150800421008210920C006FEF7E2FD20210920C00674
S31508004220FEF7DDFD43E020212348FEF7CDFD0028FB
S3150800423015D02249C868FF21F531FDF76BFBC00789
S31508004240C00F002805D110210920C006FEF7C7FDBA
S3150800425022E010210920C006FEF7BFFD1CE0174921
S31508004260C868CD21FDF756FBC007C00F002805D149
S3150800427010210920C006FEF7B2FD0DE00F49C868F7
S31508004280CD21FDF747FBC007C00F002804D0102139
S315080042900920C006FEF7A1FD08210920C006FEF781
S315080042A09EFD20210920C006FEF799FD00BF00BF2C
S315080042B010BD0000CC020020000400488401002044
S315080042C010B5B348807A030000F0D1F9050445809B
S315080042D0D4FDFC00AE48C089FF217731884203DB54
S315080042E00121AB48817235E0A948C089FF217331A5
S315080042F088420ADAA64878384088022805D002217A
S31508004300A3487838418000F07DF92021A148FEF7BE
S315080043105BFD00281ED0A049C868FF21F531FDF7CE
S31508004320F9FAC007C00F002805D110210920C006D8
S31508004330FEF755FD04E010210920C006FEF74DFDE5
S3150800434020210920C006FEF74AFD08210920C006DB
S31508004350FEF745FD1AE18E48C089FF219A31884249
S3150800436003DB02218A4881722FE020218948FEF763
S315080043702BFD002829D08849C868FF21F531FDF7AB
S31508004380C9FAC007C00F002805D108210920C006B0
S31508004390FEF725FD04E008210920C006FEF71DFDED
S315080043A010210920C006FEF71AFD20210920C006A3
S315080043B0FEF715FD764878384088012805D0012192
S315080043C073487838418000F01DF9DFE07048C089ED
S315080043D0FF21B331884203DB03216D48817248E02F
S315080043E020216C48FEF7F0FC002842D0FF2101315D
S315080043F06848FEF7E9FC002807D06748006A67495D
S31508004400884202D90421624881726349C868FF213B
S31508004410F531FDF77FFAC007C00F00280FD110212C
S315080044200920C006FEF7D9FC08210920C006FEF7B8
S31508004430D4FC20210920C006FEF7CFFC0EE010218F
S315080044400920C006FEF7CBFC20210920C006FEF78E
S31508004450C6FC08210920C006FEF7C1FC4C4878387E
S315080044604088002805D0002149487838418000F066
S31508004470C9F88BE020214748FEF7A6FC002845D05E
S31508004480FF2101314348FEF79FFC002807D0424828
S31508004490006A4249884202D904213D4881723E4950
S315080044A0C868FF21F531FDF735FAC007C00F0028A7
S315080044B012D110210920C006FEF78FFC0821092019
S315080044C0C00601E061E022E0FEF787FC2021092012
S315080044D0C006FEF782FC0EE010210920C006FEF792
S315080044E07EFC20210920C006FEF779FC0821092058
S315080044F0C006FEF774FC264878384088002805D0A0
S31508004500002123487838418000F07CF83EE02021DD
S315080045102048FEF759FC002836D01D4878384088D0
S31508004520002805D000211A487838418000F06AF83A
S315080045301948C0691A4988420FD210210920C006B5
S31508004540FEF74BFC08210920C006FEF746FC202191
S315080045500920C006FEF741FC0EE010210920C0061E
S31508004560FEF73DFC20210920C006FEF738FC08218D
S315080045700920C006FEF733FC074838304078012882
S3150800458002D103210248817200E000BF00BF10BDBE
S315080045904403002000040048840100209411000010
S315080045A03075000010B5FEF725FAFEF781F901F01F
S315080045B075FD10BD034880684008400001498860C1
S315080045C070470000002C004003488068002801D08E
S315080045D0012070470020FCE7002C004010B5FFF7CB
S315080045E0F3FF002804D0FFF7E5FF662000F002F885
S315080045F010BD00004106490E014A116070470000CF
S31508004600002C004010B57E20FFF7F4FF0948FEF79E
S3150800461069FA0949094801810621083000F0C2F8FB
S315080046200649083188814022024904480830FEF7C5
S3150800463096FA10BD00F80008FBAA0000C402002084
S315080046402021020C01D010211046020A01D0104682
S315080046500839020901D01046091F820801D0104600
S31508004660891E420801D0881E7047081A704730B460
S315080046707446641E2578641CAB4204D3635D5B00F4
S31508004680E31830BC18471D46F8E7000010B50028A7
S3150800469019DB1A4A03231B02D21883089B00D25837
S315080046A08307DC0EFF23A3409A438B071B0E840760
S315080046B0E40EA3401A43114B032424021B19840851
S315080046C0A4001A5118E00E4A03071B0F083B9B0863
S315080046D09B00D2588307DC0EFF23A3409A438B071F
S315080046E01B0E8407E40EA3401A43054B0407240F48
S315080046F0083CA408A4001A5110BD000000E100E01F
S315080047001CED00E002E008C8121F08C1002AFAD111
S3150800471070477047002001E001C1121F002AFBD133
S315080047207047000010B51948007801282DD10020DF
S31508004730164908701649088012E015480088400096
S315080047401449085A14490988C900144A8918104A8C
S315080047501288520088520E480088401C0C4908806E
S315080047600B4800880428E8DB7E20FFF743FF0A4849
S315080047700088401C0849088008460088142804DB7D
S315080047800020088001200649087010BD6401002039
S315080047907A010020F00300207C0100202804002074
S315080047A05C01002010B502460023002901D1002033
S315080047B010BD03E01488921CE01883B208464C1E0C
S315080047C0A1B20028F6D11846F2E7000070B5002518
S315080047D0AF48807A01280ED1AD483838C06AFF2123
S315080047E0F531884207D90021A94881720020A949D4
S315080047F00880A9490870A648407A012872D1A548B8
S31508004800007A012811D003280ED1A448007E00287A
S3150800481006D19F48007A002802D101219C480172DE
S3150800482000209B49383948612CE19A48407A082883
S315080048307DD007DC0300FFF71AFF08142558867E8B
S315080048409D9EAE7EA52873D006DC092871D00A285D
S3150800485070D0A1286FD103E1AA286DD0AB28F9D171
S3150800486008E100208A493839486101218848C17120
S31508004870002202218A48FFF78CFB00208449383938
S31508004880C860FDE000208249383948618148807A4D
S31508004890012811D17F48007B282825DA7D48007B2E
S315080048A00A2821DD7B48017B7948103041810121A6
S315080048B010388173C17017E07648807A022812D1C1
S315080048C0744A117BD07A00F06BFE0546282D0BDA68
S315080048D00A2D09DD6E481030458101211038817393
S315080048E0C17001E0D2E070BDCAE0002068493839DD
S315080048F048616848807A022824D1664A117BD07AB2
S3150800490000F04EFE012803D103216448017619E020
S31508004910604A117BD07A00F043FE002812D10021AC
S315080049205E4801765A48C07B01280BD105E042E073
S3150800493099E048E08EE0A2E098E000F037FD00211B
S315080049405348C1739CE05348807A02280ED1514AD5
S31508004950117BD07A00F024FE4D491031C880012120
S315080049604B48C173002001F0CDF802E0012001F0A8
S31508004970C9F885E084E00020454938394861454A48
S31508004980117BD07A00F00CFE414910314880012095
S3150800499001F05AF974E000203D49383948613D4A2A
S315080049A0117BD07A00F0FCFD39491031888003204C
S315080049B001F04AF964E00020354938394861022097
S315080049C001F042F95CE00020314938394861314943
S315080049D0887AC117890F091889108900411A33D1B5
S315080049E02C49887AC117890F09188910284A103264
S315080049F01181104600891C2826DA00241FE0A2002F
S31508004A00921D244B9B1D995CA200521D985C00F0D8
S31508004A10C7FD0146A2001E481E308152A200083278
S31508004A201C4B9B1D995CA200D21D985C00F0B8FD3A
S31508004A300146A20016481E3010184180641C14480E
S31508004A4010300089A042DADC042001F0FDF800F0FD
S31508004A50ADFC15E0052001F0F7F800F0A7FC0FE023
S31508004A6001F0B8F80CE000F0E9FF09E001210B4875
S31508004A70C17605E0012109482030817100E000BFB8
S31508004A8000BF00BF00BF00210148417200BF2AE7EE
S31508004A90BC010020C8040020810100204403002036
S31508004AA00038014070B505460C46002D02D0012D90
S31508004AB01ED10CE0602101208007FFF73BF9002199
S31508004AC001208007FFF798F90A48047010E00948A2
S31508004AD00078A04209D0602101208007FFF72AF953
S31508004AE0214601208007FFF787F90248047000BFB6
S31508004AF000BF70BD7F01002010B5F848007A012874
S31508004B007ED1F748007E0028FAD1F448407A03009F
S31508004B10FFF7ADFD08050765C1EFEEEDECEB0020EC
S31508004B2010BDEF492039C868FF219131FCF7F2FE24
S31508004B308007800F00280AD110210920C006FEF739
S31508004B404EF908210920C006FEF749F940E0E44974
S31508004B502039C868FF219131FCF7DCFE8007800FF9
S31508004B6001280AD110210920C006FEF736F90821C6
S31508004B700920C006FEF733F92AE0D9492039C86862
S31508004B80FF219131FCF7C6FE8007800F02280AD163
S31508004B9010210920C006FEF722F908210920C006BF
S31508004BA0FEF71DF914E0CE492039C868FF21913176
S31508004BB0FCF7B0FE8007800F032809D108210920D9
S31508004BC0C006FEF70AF910210920C006FEF707F904
S31508004BD020210920C006FEF702F90120A0E7C049F6
S31508004BE02039C868C821FCF795FE8007800F002881
S31508004BF00CD110210920C006FEF7F1F8082100E0C3
S31508004C008BE10920C006FEF7EAF83DE0B4492039F1
S31508004C10C868C821FCF77EFE8007800F01280AD1E4
S31508004C2010210920C006FEF7D8F808210920C00679
S31508004C30FEF7D5F828E0AA492039C868C821FCF744
S31508004C4069FE8007800F02280AD110210920C006B4
S31508004C50FEF7C5F808210920C006FEF7C0F813E0DC
S31508004C609F492039C868C821FCF754FE8007800F81
S31508004C70032809D108210920C006FEF7AEF810213D
S31508004C800920C006FEF7ABF820210920C006FEF76A
S31508004C90A6F8012044E792492039C868C821FCF7DC
S31508004CA039FE8007800F00280AD110210920C00686
S31508004CB0FEF795F808210920C006FEF790F842E0AD
S31508004CC087492039C868C821FCF724FE8007800F69
S31508004CD001280FD110210920C006FEF77EF8082109
S31508004CE00920C006FEF77BF82DE015E1E6E08BE02B
S31508004CF05DE02FE07A492039C868C821FCF70AFE2A
S31508004D008007800F02280AD110210920C006FEF765
S31508004D1066F808210920C006FEF761F813E0704915
S31508004D202039C868C821FCF7F5FD8007800F0328DD
S31508004D3009D108210920C006FEF74FF810210920DD
S31508004D40C006FEF74CF820210920C006FEF747F8F2
S31508004D500120E5E662492039C868FF212D31FCF7B4
S31508004D60D9FDC007C00F002805D110210920C006AB
S31508004D70FEF735F80FE05A492039C868FF212D316A
S31508004D80FCF7C8FDC007C00F002804D01021092071
S31508004D90C006FEF722F820210920C006FEF71FF8F4
S31508004DA008210920C006FEF71AF80120B8E64C4982
S31508004DB02039C868FF219131FCF7ACFDC007C00F48
S31508004DC0002805D110210920C006FEF708F80FE0D3
S31508004DD043492039C868FF219131FCF79BFDC0077C
S31508004DE0C00F002804D010210920C006FDF7F5FFE2
S31508004DF020210920C006FDF7F2FF08210920C00678
S31508004E00FDF7EDFF01208BE635492039C868C82132
S31508004E10FCF780FD8007800F00280AD110210920A1
S31508004E20C006FDF7DCFF08210920C006FDF7D7FFFD
S31508004E303DE02B492039C868C821FCF76BFD80077F
S31508004E40800F01280AD110210920C006FDF7C5FFE9
S31508004E5008210920C006FDF7C2FF28E020492039AD
S31508004E60C868C821FCF756FD8007800F02280AD1BA
S31508004E7010210920C006FDF7B2FF08210920C00647
S31508004E80FDF7ADFF13E016492039C868C821FCF7BD
S31508004E9041FD8007800F032809D108210920C00693
S31508004EA0FDF79BFF10210920C006FDF798FF20217A
S31508004EB00920C006FDF793FF012031E6084920398D
S31508004EC0C868C821FCF726FDC007C00F002809D10D
S31508004ED010210920C006FDF782FF11E044030020D7
S31508004EE0A40100200E49C868C821FCF713FDC007B5
S31508004EF0C00F002804D010210920C006FDF76DFF59
S31508004F0020210920C006FDF76AFF08210920C006EE
S31508004F10FDF765FF012003E600BF00BF00E60000BD
S31508004F208401002010B5F648007E002833D0F548E5
S31508004F30C07801282FD1F3483838C068F24988422A
S31508004F400ED9EF48008A64280ADAED48407A002824
S31508004F5006D10721EA4841720020EA493839C86073
S31508004F60E748007E032816D0E548008AFF21EB3182
S31508004F70884210DDE248407A00280CD1E1483838EA
S31508004F80C068E249884206D90321DD4841720020FB
S31508004F90DC493839C860DA48007A01286FD1D84820
S31508004FA0407A0300FFF763FB080507427EB8F7EF70
S31508004FB0EEED002010BDD3483838C068E121C9009D
S31508004FC088422DD908210920C006FDF708FF2021AF
S31508004FD00920C006FDF703FF10210920C006FDF7CA
S31508004FE0FEFE0121C7481838017618308079002856
S31508004FF007D1C4493839C8600021C14801724172D5
S315080050000AE0C0483838C068AF210901884203D988
S315080050100020BC493839C8600121BA48417103E00B
S315080050200021B848183801760120C3E7B548383852
S31508005030C068B74988422FD908210920C006FDF75C
S31508005040CEFE20210920C006FDF7C9FE1021092041
S31508005050C006FDF7C4FE0121AA48183801761830A3
S31508005060807900280CD1A7493839C8600021A4489E
S31508005070017241720020A3493839C86010E03DE149
S31508005080A0483838C068AF210901884208D90020ED
S315080050909C493839C86003E000219A4818380176D7
S315080050A0012087E797483838C0689A4988422DD939
S315080050B008210920C006FDF792FE20210920C00616
S315080050C0FDF78DFE10210920C006FDF788FE012197
S315080050D08C48183801761830807900280BD1894910
S315080050E03839C86000218648017241720020854916
S315080050F03839C8600EE083483838C068864988421F
S3150800510008D900207F493839C86003E000217D4866
S315080051101838017601204DE77A483838C0687D216D
S315080051200901884231D908210920C006FDF757FE32
S3150800513020210920C006FDF752FE10210920C006CD
S31508005140FDF74DFE01216F48183801761830807931
S3150800515000280BD16B493839C860002168480172AC
S315080051604172002067493839C86012E06548383806
S31508005170C068664988420CD9002062493839C86037
S3150800518007E0BAE07EE042E005E000215D48183815
S31508005190017601200EE75B483838C068E121C9006E
S315080051A088422ED908210920C006FDF718FE2021BD
S315080051B00920C006FDF713FE10210920C006FDF7D9
S315080051C00EFE01214F4818380176183080790028DC
S315080051D00BD14C493839C8600021494801724172DF
S315080051E0002048493839C8600FE046483838C06852
S315080051F0AF210901884208D9002042493839C860D8
S3150800520003E000213F48183801760120D2E63D48E0
S315080052103838C0684049C83988422DD9082109203C
S31508005220C006FDF7DCFD20210920C006FDF7D7FDE5
S3150800523010210920C006FDF7D2FD01213148183892
S3150800524001761830807900280BD12E493839C86084
S3150800525000212B480172417200202A493839C8605A
S315080052600EE028483838C0682C49884208D90020FA
S3150800527024493839C86003E00021224818380176E5
S31508005280012097E61F483838C068214988422ED938
S3150800529008210920C006FDF7A2FD20210920C00625
S315080052A0FDF79DFD10210920C006FDF798FD012197
S315080052B01448183801761830807900280BD111491E
S315080052C03839C86000210E480172417200200D4924
S315080052D03839C8600FE00B483838C0680D49C831FE
S315080052E0884208D9002007493839C86003E00021F8
S315080052F004481838017601205CE600BF00BF59E66D
S3150800530044030020BC010020204E0000B80B00001A
S31508005310A4060000C4090000AC0D0000CC10000073
S3150800532010B5052416E0FF2101311F48FCF735FBAF
S31508005330FF2101311C48FDF73BFAFE211A48FDF70B
S3150800534039F901461848C030C08F814202D100F0B1
S3150800535057FB10BD2046611ECCB20028E3D10524B8
S3150800536016E0FF2101311048FCF717FBFF21013138
S315080053700D48FDF73BFAFE210B48FDF71BF90146E0
S315080053800948C030C08F814202D100F039FBE0E7FE
S315080053902046611ECCB20028E3D100F02BF900F0BC
S315080053A005F800BFD5E70000CC01002010B5FDF7D1
S315080053B083FB1A491A480181083000891C2815DA26
S315080053C01748083001890E30FDF76EF81449083180
S315080053D0088908E00022830011491631CA52830061
S315080053E059184A80401C1E28F4D300E010BDFE213F
S315080053F00B480830FDF7DEF801460948C830C18772
S31508005400FF210131C038FDF72DFAFF21013104488B
S315080054100830FDF733FA00BFE8E70000FBAA0000F2
S31508005420C401002070B5044600250121594881723F
S31508005430002058493839C86257480088FA2804DDD8
S3150800544000205549088055490870544800780300DB
S31508005450FFF70DF908051D2B3F4B586D799CAA2CB3
S315080054600DD101204D4908704B4801880088401C21
S31508005470494A1080901D445400201146C870BB2C20
S3150800548004D101210920C006FDF7A7FC7FE0FB2C0B
S315080054900AD1414801880088401C3F4A1080901D67
S315080054A0445402203D49087071E0012C03D10320C1
S315080054B03A49087004E0032C02D1062037490870DF
S315080054C0354801880088401C334A1080901D445492
S315080054D05DE0314801880088401C2F4A1080901DE5
S315080054E0445404202D49087051E02B4884700188E3
S315080054F00088401C284A1080901D445405202749DE
S31508005500087044E02448C078401CC0B22249C870DC
S315080055108978884202DB0620204908701E480188DF
S315080055200088401C1C4A1080901D44542FE01A48DD
S3150800553001880088401C184A1080901D4454072092
S315080055401649087023E0144801880088401C124A4E
S315080055501080901D4454801F0188801DFDF72AF88D
S31508005560002809D100210B488172012141720020CF
S315080055700A4908700849088007480088FA2804DD9F
S315080055800020054908800549087000E000BF00BFF3
S3150800559070BD0000BC010020C80400208101002065
S315080055A070B50246002013460C461D02FF26360239
S315080055B035402543284670BD00BF00BF00BF00BF69
S315080055C000BF00BF00BF00BF00BFFEE7074908488D
S315080055D001810021083041805F21C900C180152161
S315080055E081805F210181002141817047FBAA00006B
S315080055F0C402002000201D4A1D490A81F0220831F4
S315080056004A8014228A8002220A8119224A81194A6A
S315080056108A819200CA8000BF0FE0002283001449E5
S315080056208E31CA52830059184A80830010491631B0
S31508005630CA52830059184A80401C1C28EDDB0022F8
S315080056400B490831CA81FF225F320A8214224A8234
S31508005650FF225F328A8200228031CA80891D4A80F1
S3150800566014228A80FF225F32CA807047FBAA000094
S31508005670C4010020EE02000010B57E20FEF7BAFF36
S31508005680FFF73AFA012800D110BD6348007A0128CD
S315080056907DD16148007E002802D0012865D13AE014
S315080056A020215E48FDF790FB002826D101215A48A3
S315080056B04176FF38C138C069594988422AD25948C3
S315080056C0C0687D210901884224D253487838408928
S315080056D0002802D1FEF7FAFC1CE010210920C006BA
S315080056E0FDF77DFB20210920C006FDF778FB082180
S315080056F00920C006FDF773FB0CE04A48406A484992
S31508005700884202D2FEF7E2FC04E0012142484176D3
S31508005710FEF7D6FD7DE04349C868FF21F531FCF761
S31508005720F9F8C007C00F00280FD110210920C006BC
S31508005730FDF753FB08210920C006FDF74EFB202183
S315080057400920C006FDF749FB0EE010210920C00616
S31508005750FDF745FB20210920C006FDF740FB08217F
S315080057600920C006FDF73BFB53E02B48007E0528C1
S315080057702BD12C49C868FF21F531FCF7CBF8C007B7
S31508005780C00F002811D110210920C00600E041E011
S31508005790FDF723FB08210920C006FDF71EFB202183
S315080057A00920C006FDF719FB32E010210920C006C2
S315080057B0FDF715FB20210920C006FDF710FB08217F
S315080057C00920C006FDF70BFB22E01348007E0628D9
S315080057D00FD110210920C006FDF701FB2021092061
S315080057E0C006FDF7FCFA08210920C006FDF7F7FAFE
S315080057F00EE010210920C006FDF7EFFA082109205E
S31508005800C006FDF7EAFA20210920C006FDF7E5FAE9
S3150800581000BF00BF00BF37E744030020000400486C
S315080058203075000084010020FEF734F9FDF7D6FD37
S3150800583008210920C006FDF7D2FA20210920C00652
S31508005840FDF7CDFA10210920C006FDF7C8FAE120B8
S315080058504002FCF759FEFDF7C3FCFCF701FFFCF715
S3150800586097FC0C20FCF702FC0920FCF7FFFB08203C
S31508005870FCF7FCFB0720FCF7F9FB01214648FCF77F
S315080058802DFD01214548017200214172FF388938F2
S3150800589041718171012141484173FDF7D3FCFEF73F
S315080058A041F93F496320FEF793F91A216320FEF771
S315080058B0E3F9FFF735FDFEF7EDFA00F07BF8374818
S315080058C078384089002801D1FEF700FC00213548C8
S315080058D0417040213448FDF782FAFEF763FE002145
S315080058E03048C171FDF7FEFD01210920C006FDF70C
S315080058F076FA4FE02B48C079002802D0012844D117
S315080059000AE0FEF763FFFCF711FDFFF7B5FEFDF7AA
S3150800591099FC00F0E9FB3CE00021084600F0FCF9A0
S3150800592020483838C0682149884208D900211D48CE
S31508005930C171012202211E48FEF72BFB1FE01949FF
S315080059403839C868FF21F531FBF7E4FFC007C00FF7
S3150800595000280FD110210920C006FDF740FA2021A2
S315080059600920C006FDF73BFA08210920C006FDF705
S3150800597036FA04E020210920C006FDF72EFAFCF7C6
S315080059803FFD7E20FEF736FE03E000210548C17183
S3150800599000BF00BFAEE7000000240140440300201A
S315080059A0581B0000BC01002000040048204E0000DF
S315080059B00038014010B540210F48FBF7EEFF4021A3
S315080059C00D48FCF731FF06210B48FEF7EBFE0A49A6
S315080059D0898988420AD108480838008907498842CF
S315080059E008D0FFF7F3FDFEF70DFE03E0FFF7EEFD27
S315080059F0FEF708FE10BD0000CC020020FBAA00003E
S31508005A0010B500240C484089052803DB0A4840895C
S31508005A10282803DD19210848418101240648008900
S31508005A201D2803DD0124022103480181012C01D12F
S31508005A30FFF7BCFC10BD0000CC01002070B5A0B07B
S31508005A400025002680216846FBF7A7FFAA2168469D
S31508005A500170FB21417001218170A521C170124896
S31508005A60007A8006010E6846017102790E490E31E8
S31508005A70401DFBF779FF68460079411D6846FCF72B
S31508005A8099FD0446211268460079401D6A4611545C
S31508005A9068460079801D145468460079C11D684619
S31508005AA0FEF74CFA20B070BDCC01002030B5A1B08D
S31508005AB00446802101A8FBF770FF0025AA21684645
S31508005AC00171FB214171022181710121C1710221FC
S31508005AD00172FF200002204001126846417284725A
S31508005AE0072101A8FCF766FD0546FF2000022840AD
S31508005AF001126846C1720573092101A8FEF71EFA4C
S31508005B0021B030BD30B5A1B00446802101A8FBF70D
S31508005B1044FF0025AA2168460171FB214171012134
S31508005B208171A621C17102210172FF200002204065
S31508005B300112684641728472072101A8FCF73AFDF2
S31508005B400546FF200002284001126846C172057307
S31508005B50092101A8FEF7F2F921B030BDF0B585B0EC
S31508005B6004460D46164600200090019002900390C8
S31508005B700027AA2168460170FB2141700121817026
S31508005B80A721C17002210171FF20000220400112E5
S31508005B90684641718471FF20000228400112684658
S31508005BA0C1710572FF200002304001126846417239
S31508005BB086720B21FCF7FEFC0746FF2000023840E0
S31508005BC001126846C17207730D21FEF7B7F905B0D1
S31508005BD0F0BD0000F0B5A1B000260027802101A87D
S31508005BE0FBF7DBFE0025AA2168460171FB214171FE
S31508005BF001218171A121C1710B2101720FA5027AC0
S31508005C0029460930FBF7B0FE6846007A411D01A80F
S31508005C10FCF7D0FC044621126846007A401D01AA0A
S31508005C2011546846007A801D14546846007AC11DCE
S31508005C3001A8FEF783F921B0F0BD00004E5F43329C
S31508005C4043355F56315F330030B5A1B00446802135
S31508005C5001A8FBF7A2FE0025AA2168460171FB21CF
S31508005C604171022181710521C17102210172FF2052
S31508005C70000220400112684641728472072101A879
S31508005C80FCF798FC0546FF200002284001126846EA
S31508005C90C1720573092101A8FEF750F921B030BD7C
S31508005CA0F0B585B004460D461646002000900190D2
S31508005CB0029003900027AA2168460170FB214170D3
S31508005CC001218170A821C17003210171FF20000202
S31508005CD028400112684641718571FF200002204064
S31508005CE001126846C1710472FF2000023040011299
S31508005CF06846417286720B21FCF75CFC0746FF205A
S31508005D000002384001126846C17207730D21FEF77A
S31508005D1015F905B0F0BD000070B504460D4600261D
S31508005D20002D13D10846FEF7BDFE0021D448818216
S31508005D30FF38893841730020D2498862D2490870F1
S31508005D40D04908630021CE48C18297E1CD48383052
S31508005D50407B002877D1CB48806AFF21F5318842FD
S31508005D6072D90020C7498862C548018A601F8142E6
S31508005D700EDDC5480078C54908600221C14838309B
S31508005D804173BF48018A81827D20C000C0490880CE
S31508005D90BB48818A008A81420BDD0121B948383027
S31508005DA04173B748018A81827D20C000B8490880BE
S31508005DB00EE0B348018A20461430814208DDB24815
S31508005DC000780F2804DDB0480078401FAE490870F7
S31508005DD0AB48018A20463738814236DAA8487838EF
S31508005DE04088002803D14820A749087010E0A44835
S31508005DF078384088012803D15120A349087007E064
S31508005E009F4878384088022802D15A209E4908704F
S31508005E109C48006B9F49884230D9002099490863FD
S31508005E209748C18A008A814209DB9548407A00284A
S31508005E3005D107219248417200209249C8609048CE
S31508005E40018AC1821AE022E01BE08D48018A2046B9
S31508005E502638814209DD8C4800780F280EDD8A48ED
S31508005E600078801E8849087008E0874800780F285F
S31508005E7004DD85480078C01E834908708048018A79
S31508005E808182814801780120FEF70CFEF6E07D4804
S31508005E903830407B01287CD17A48806A7C49098859
S31508005EA0884262D90020774988627548818A008AC3
S31508005EB081425BDA7248018A20461438814215DA33
S31508005EC0FF20F530724908806D48018A808A081AD1
S31508005ED0042805DA6C480078801C6B49087035E0A0
S31508005EE069480078401C684908702FE06448018AB0
S31508005EF020460A38814215DAFF20F53064490880C1
S31508005F005F48018A808A081A022805DA5E480078FE
S31508005F10401C5D49087019E05B480078801E5A49A4
S31508005F20087013E05648018A601F81420EDAFF2086
S31508005F30F530574908805248018A808A081A02288B
S31508005F4004DB51480078801E4F4908704C48018A86
S31508005F508182008AA04256DD7D20C0004C49088017
S31508005F6049480078801E484908704CE04448008A31
S31508005F70A04219DD4248008A001B05280ADD7D205B
S31508005F80C0004349088040480078801E3E49087092
S31508005F9036E04DE07D20C0003D4908803A4800784B
S31508005FA0401E394908702BE03548008AA04227D0A0
S31508005FB03348018A808A081A032805DD32480078A2
S31508005FC0801C314908701BE02D48018A2046083894
S31508005FD0814209DAAF2080002D4908802A480078D6
S31508005FE0C01C294908700BE02B4829490880244819
S31508005FF0008AA04204DA24480078801C22490870E6
S315080060001F48018A8182204800780A2803DA0A2074
S315080060101D49087006E01C4800783C2802DD3C2033
S3150800602019490870184801780120FEF73BFD25E05C
S3150800603015480078282804DD1348007810381249D6
S3150800604008700F48018AE01C814204DC0C48018A6A
S31508006050E01E81420ADA01210A48383041730848AD
S31508006060018A81827D20C000094908800448018A86
S315080060708182054801780120FEF714FD70BD0000F5
S315080060804403002084010020FE000020C8000020F0
S3150800609000010020B80B0000DC05000008B501214E
S315080060A04804FDF73DFA01218804FDF739FA6846E8
S315080060B0FCF797FE0421684601804821C1706946AD
S315080060C00920C006FCF7EAFD6846FCF78AFE20218F
S315080060D0684601800421C17069460248FCF7DEFD66
S315080060E008BD00000004004870B50024FEF71AFF3A
S315080060F001280CD1FE48C068FF21F531884205D930
S315080061000121C9030920C006FCF767FE70BDF948DE
S31508006110007A00287CD10121F64841760020F6490C
S31508006120087000210846FFF7F7FD0021F0483830CF
S31508006130C1701838017608210920C006FCF74FFE01
S3150800614020210920C006FCF74AFE10210920C006B6
S31508006150FCF745FE0021E7480176E548C068FF21BF
S31508006160F531884209D2E24838304079002803D10F
S315080061700121DF483830C172CFE10021DC483830D0
S3150800618041713838C068DD49884232D9D948407BE0
S3150800619000280FD1D648C0687D214901884201D21E
S315080061A0FDF752FF0021D34841727D204001D049B6
S315080061B0C8600CE0CF48007B012808D10020CC49F4
S315080061C0C8600021CB484172017601210172202165
S315080061D0CB48FCF7F9FD002805D00021C548017613
S315080061E00121017299E101210920C006FCF7F5FD9C
S315080061F093E1C048007B0128BED10020BC49C86095
S315080062000021BC48417201760121017285E1FFE750
S31508006210B848007E01280BD0B648007E022807D071
S31508006220B448007E052803D0B248007E03282ED144
S31508006230B048C07E01282AD1AD49C8687D21C90069
S31508006240FBF768FB002918D1A948C168FF308130DF
S3150800625001664030007F00280FD1A549C8687D2116
S31508006260C900FBF757FB85B2A248828C018A2846EB
S31508006270FFF716FD01219F4801779D48C168FF3049
S315080062808130006E081A02D000219A480177994891
S31508006290007E0300FEF7EBF907055F80A2ACB5EFB9
S315080062A05E0000210846FFF737FD91483830807BAD
S315080062B0002804D100218E483830C17003E001213E
S315080062C08B483830C1708A483830C07B012805D1E0
S315080062D0FFF76CF8002186483830C1738448C068D7
S315080062E07D210901884226D9002083490870804803
S315080062F03830007A00282DD120218148FCF764FD2A
S31508006300002814D108210920C006FCF768FD2021C1
S315080063100920C006FCF763FD10210920C006FCF71A
S315080063205EFD01210920C006FCF757FD12E000209A
S315080063306F49C8600EE06E48C068FF21F531884293
S3150800634008D96C4878384089002803D10021684864
S315080063503830C172E0E00121654838304170C170BB
S315080063606349C8687D21C900FBF7D4FA60494831FA
S315080063708988884206D902215E4801760121FF38BC
S315080063808938C1725A49C86800F0DAF8044601210A
S315080063902046FFF7C1FCBFE001215548383041705F
S315080063A0C1705349C86800F0CBF80446012120465D
S315080063B0FFF7B2FC4E49C8687D21C900FBF7AAFA67
S315080063C04B49483149880F39884206D9012148483E
S315080063D03830C1720521474801769DE001214448BD
S315080063E038304170C170FF208730FFF795FC93E085
S315080063F001213F483830C17000210846FFF78CFC60
S315080064008AE001213B484176FF388938C17038381F
S31508006410C16848304088401E7D22D2005043FF3074
S31508006420F530814209D23249C86800F089F8044635
S3150800643001212046FFF770FC44E000210846FFF7DB
S315080064406BFC01212A483830C1723838C168483097
S315080064504088401E7D22D2005043AF229200801809
S3150800646081422FD3224838308079012804D1062169
S315080064702048017620E026E020212148FCF7A4FCEC
S31508006480002816D108210920C006FCF7A8FC2021FF
S315080064900920C006FCF7A3FC10210920C006FCF75A
S315080064A09EFCFDF7D1FD01210920C006FCF795FCED
S315080064B002E000210F4801760121C9030920C00620
S315080064C0FCF78BFC28E00B48407A002823D10848C3
S315080064D0C0680C4988421ED9FDF7B6FD002004495C
S315080064E0C860044878384088032810DA01210BE090
S315080064F08401002044030020C4000020B80B0000DB
S3150800650000040048102700000B48017603E000212C
S3150800651009480176017200BF00BF08484068FF219C
S31508006520F531884202D90020044948607E20FEF7EA
S3150800653061F800BFEAE5000044030020840100205A
S31508006540F8B5054600247D21C9002846FBF7E2F97F
S31508006550064600270020009000BF0BE0A1000C486B
S31508006560405AB04205DCA100094808184088009046
S315080065700127641C06480E380089A042EEDC002F6D
S3150800658003D103480E38008A00900098F8BD000031
S31508006590DA01002000C1814001C0804101C080416C
S315080065A000C1814001C0804100C1814000C18140D5
S315080065B001C0804101C0804100C1814000C18140C5
S315080065C001C0804100C1814001C0804101C08041B5
S315080065D000C1814001C0804100C1814000C18140A5
S315080065E001C0804100C1814001C0804101C0804195
S315080065F000C1814000C1814001C0804101C0804185
S3150800660000C1814001C0804100C1814000C1814074
S3150800661001C0804101C0804100C1814000C1814064
S3150800662001C0804100C1814001C0804101C0804154
S3150800663000C1814000C1814001C0804101C0804144
S3150800664000C1814001C0804100C1814000C1814034
S3150800665001C0804100C1814001C0804101C0804124
S3150800666000C1814001C0804100C1814000C1814014
S3150800667001C0804101C0804100C1814000C1814004
S3150800668001C0804100C1814001C0804101C08041F4
S3150800669000C1814000C0C101C30302C2C60607C7C4
S315080066A005C5C404CC0C0DCD0FCFCE0E0ACACB0B34
S315080066B0C90908C8D81819D91BDBDA1A1EDEDF1F64
S315080066C0DD1D1CDC14D4D515D71716D6D21213D354
S315080066D011D1D010F03031F133F3F23236F6F73704
S315080066E0F53534F43CFCFD3DFF3F3EFEFA3A3BFBF4
S315080066F039F9F83828E8E929EB2B2AEAEE2E2FEFA4
S315080067002DEDEC2CE42425E527E7E62622E2E32313
S31508006710E12120E0A06061A163A3A26266A6A76743
S31508006720A56564A46CACAD6DAF6F6EAEAA6A6BABB3
S3150800673069A9A86878B8B979BB7B7ABABE7E7FBFE3
S315080067407DBDBC7CB47475B577B7B67672B2B373D3
S31508006750B17170B050909151935352929656579783
S31508006760559594549C5C5D9D5F9F9E5E5A9A9B5B73
S3150800677099595898884849894B8B8A4A4E8E8F4F23
S315080067808D4D4C8C44848545874746868242438393
S3150800679041818040B4670008C8000020BC000000A2
S315080067A00447000870680008840100204C080000AF
S315080067B01447000800000000000000000000000068
S315080067C000000000000000000000000000000000BB
S315080067D000000000000000000000000000000000AB
S315080067E0000000000000000000000000000000009B
S315080067F00000000001020304010203040607080959
S3150800680000A24A0400000000000000000102030480
S31508006810060708090000000000000000000000004C
S315080068200000000000000000040000000100000055
S31508006830000000000000000000000000000000004A
S31508006840000000000000000000000000000000003A
S31508006850000000000000000000000000000000002A
S31508006860000000000000000000000000000000001A
S705080018C515
